:1000000002006EC0E0C083C082C0D075D000C007BF
:10001000AFBA43BA8090FE53E030E004E4F0C20986
:1000200090FA72E030E031300A09C20A90FA71E4C5
:10003000F08020900213E024FFF0900212E034FFE1
:10004000F0E07002A3E090FA717005F0D2B4800382
:1000500074A0F090FA72E4F08FBAD007D0D0D082BA
:05006000D083D0E03266
:10006B00020003787FE4F6D8FD7581210200B5020A
:10007B0011FDE493A3F8E493A34003F68001F20887
:10008B00DFF48029E493A3F85407240CC8C333C4CA
:10009B00540F4420C8834004F456800146F6DFE435
:1000AB00800B01020408102040809011CDE47E01EA
:1000BB009360BCA3FF543F30E509541FFEE493A3A8
:1000CB0060010ECF54C025E060A840B8E493A3FABA
:1000DB00E493A3F8E493A3C8C582C8CAC583CAF046
:1000EB00A3C8C582C8CAC583CADFE9DEE780BE9054
:1000FB0002187401F090021D74FFF090021B740043
:10010B00F0A37400F09002197402F0A37402F07B58
:10011B00017A027918120F67E4FBFD7F01020FB120
:02012B0021DDD4
:0201330021DDCC
:02013B0021DDC4
:0201430021DDBC
:02014B0021DDB4
:0201530021DDAC
:02015B0021DDA4
:020163008078A2
:02016B008070A2
:020173008068A2
:02017B008060A2
:020183008058A2
:02018B008050A2
:020193008048A2
:02019B008040A2
:0201A3008038A2
:0201AB008030A2
:0201B3008028A2
:0201BB008020A2
:0201C3008018A2
:0201CB008010A2
:0201D3008008A2
:1001DB008000016BE5082425F582E43402F583E009
:1001EB00050822900222300703900225E475F001E6
:1001FB001208FA0208542000E97F2ED2008018EF73
:10020B00540F2490D43440D4FF30040BEF24BFB4EC
:10021B001A0050032461FFE50960021509050CE57E
:10022B000C7002050B30070E900222E475F00112E0
:10023B0008FAEF0208E802110D7403D2078003E4F9
:10024B00C207F508900222120911E4F509F50BF526
:10025B000CE50960077F2012022280F5750AFFC2A8
:10026B0001C200C202C203C205C206C2081201EEDD
:10027B00FF700D3007057F00120233AF0CAE0B225F
:10028B00B4255FC2D5C2041201EEFF24D0B40A001C
:10029B00501A75F00A780930D50508B6FF0106C665
:1002AB00A426F620D5047002D20380D924CFB41A29
:1002BB0000EF5004C2E5D204020434D20180C6D24E
:1002CB000080C0D20280BCD2D580BAD20580B47F68
:1002DB00201202222002077401B5090040F112011D
:1002EB00DFFF12022202025CD208D20680951201B5
:1002FB00DFFB1201DFFA1201DFF94A4B70067905B9
:10030B007A057BFF20022EE509602A7E008E82751E
:10031B00830012086D60060EEE650A70F0C2D5EB15
:10032B00C0E0EAC0E0E9C0E0EE12047BD0E0F9D017
:10033B00E0FAD0E0FB120854FF60AAEBC0E0EAC081
:10034B00E0E9C0E0120222D0E02401F9D0E0340051
:10035B00FAD0E0FBE50A0460DCD50AD980877BFF85
:10036B007A047977D202809C791080027908C206D0
:10037B00C2088008D2D5790A8004790AC2D5E50A69
:10038B00047002F50AE4FAFDFEFF1201DFFC7B08A4
:10039B002001131201DFFD7B1030000A1201DFFE7A
:1003AB001201DFFF7B20EC3382D592D55013C3E4CF
:1003BB003000069FFFE49EFEE42001039DFDE49CBC
:1003CB00FCE4CBF8C201EC700CCFCECDCCE824F81A
:1003DB00F870F38017C3EF33FFEE33FEED33FDEC14
:1003EB0033FCEB33FB994002FB0FD8E9EB300105F3
:1003FB00F8D0E0C448B201C0E00AEC4D4E4F782073
:10040B007B0070C2EAB50A0040BCC0E012047DD08C
:10041B00F0D0E0200104C4C0E0C4B201C0F012026D
:10042B000BD0F0D5F0EB02025C12091A02F9530360
:10043B00735802CA4C02C64203774F037F44037FB3
:10044B004902DF4303855503694603694503694741
:10045B0005255002CE2D02D22E02F52B02D62302F9
:10046B00F320050E2A028E48000002ED3F3F3F00AD
:10047B00790AA2D5200314300509B910020404B976
:10048B00080104A2D5200602500104200268920242
:10049B00B509005034C0E07F203003197F30A20231
:1004AB0072067205500F1204D4C202C206C205C2F4
:1004BB00087F30800F300503E9C0E01202223005BF
:1004CB0003D0E0F9D0E0B509CC3005177F30B91077
:1004DB000C1202227F583004077F788003B908037F
:1004EB001202223002057F2D0202227F202008F803
:1004FB007F2B2006F322920280CF286E756C6C291D
:10050B0000D2011201DF3001F8C201780930D501A8
:10051B0008F602028E2D504349581201DF2403B412
:10052B0005004001E490052093120213743A120265
:10053B0013D203750904020373F090022EE09002AC
:10054B003CF0900226E0FAA3E0FB900232EEF0A31F
:10055B00EFF0900236EAF0A3EBF0900234ECF0A34C
:10056B00EDF0900214E0FFA3E0900240CFF0A3EF78
:10057B00F090023AE024E0F0A3E0F9C313FF7E0011
:10058B00900232E0FAA3E02FFFEE3ACF24FFFBEF0D
:10059B0034FFFAE9FFA3E0F8A3E02FFFEE38CF24F6
:1005AB00FFCF34FF900248F0A3EFF0900232E0FE51
:1005BB00A3E0FF120EF090023CE060030206659090
:1005CB00023EF090023BE0FF90023EE0FEC39F40F4
:1005DB0003020725EF640C701790023AE075F00CDC
:1005EB00A42429F582E5F03412F583E5822E801AD6
:1005FB0090023EE0FF90023AE075F010A4249DF5C6
:10060B0082E5F03416F583E5822FF582E43583F528
:10061B0083E49390023DF0E490023FF090023BE0C4
:10062B00C313FF90023FE0C39F502690023DE03082
:10063B00E0059002368003900238E0FEA3E0FF1243
:10064B00121090023DE0C313F090023FE004F080E3
:10065B00CB90023EE004F00205CEE490023EF09017
:10066B00023BE0FF90023EE0FEC39F4003020725E2
:10067B00EF640C701790023AE075F00CA42429F586
:10068B0082E5F03412F583E5822E801A90023EE06B
:10069B00FF90023AE075F010A4249DF582E5F0344A
:1006AB0016F583E5822FF582E43583F583E4939089
:1006BB00023DF0E490023FF090023BE0C313FF9049
:1006CB00023FE0FEC39F5049900236E0FDA3E0904D
:1006DB000214CDF0A3EDF090023DE030E024EEFFEC
:1006EB00900233E02FFF900232E03400FE90023E86
:1006FB00E0FD900235E02DFD900234E03400FC1259
:10070B0010E390023DE0C313F090023FE004F08051
:10071B00A790023EE004F002066A900240E0FFA3BD
:10072B00E0900214CFF0A3EFF0900201E024FFFB66
:10073B00900200E034FFFA900217E024FFFE9002D3
:10074B0016E034FF900248F0A3CEF0E4FDFCFFFE70
:10075B00020EF0E709F608DFFA8046E709F208DF38
:10076B00FA803E88828C83E709F0A3DFFA8032E3BC
:10077B0009F608DFFA8078E309F208DFFA8070885F
:10078B00828C83E309F0A3DFFA806489828A83E099
:10079B00A3F608DFFA805889828A83E0A3F208DF88
:1007AB00FA804C80D280FA80C680D4806980F28037
:1007BB0033801080A680EA809A80A880DA80E2805D
:1007CB00CA803389828A83ECFAE493A3C8C582C8B2
:1007DB00CCC583CCF0A3C8C582C8CCC583CCDFE91C
:1007EB00DEE7800D89828A83E493A3F608DFF9ECB8
:1007FB00FAA9F0EDFB2289828A83ECFAE0A3C8C543
:10080B0082C8CCC583CCF0A3C8C582C8CCC583CC69
:10081B00DFEADEE880DB89828A83E493A3F208DFD8
:10082B00F980CC88F0EF60010E4E60C388F0ED24A8
:10083B0002B4040050B9F582EB2402B4040050AFAB
:10084B0023234582239007AE73BB010689828A83DB
:10085B00E0225002E722BBFE02E32289828A83E474
:10086B009322BB010CE58229F582E5833AF583E0FF
:10087B00225006E92582F8E622BBFE06E92582F81E
:10088B00E222E58229F582E5833AF583E49322C5DA
:10089B00F0F8A3E028F0C5F0F8E582158270021598
:1008AB0083E038F022BB0110E58229F582E5833A1B
:1008BB00F583E0F5F0A3E0225009E92582F886F0F4
:1008CB0008E622BBFE0AE92582F8E2F5F008E222EF
:1008DB00E5832AF583E993F5F0A3E99322BB01069F
:1008EB0089828A83F0225002F722BBFE01F322F8A1
:1008FB00E0FBA3A3E0F925F0F0E582158270021569
:10090B0083E0FA38F022EBF0A3EAF0A3E9F022D06F
:10091B0083D082F8E4937012740193700DA3A393A8
:10092B00F8740193F5828883E4737402936860EF23
:10093B00A3A3A380DF1211987F967E001211E67D90
:10094B00F07C787FE51211BB7D007C017F011211D9
:10095B00BB7D007C077F021211BB7D307C107F03B7
:10096B001211BBE4FDFC7F041211BB7402FDFC7F72
:10097B00081211BBE4FDFC7F091211BBE4FD7F0AD9
:10098B001211BBE4FD7F0C1211BBE4FD7F0D1211A4
:10099B00BBE4FD7F0F1211BBE4FD7F101211BB7D79
:1009AB00077F111211BBE4FD7F121211BBE4FD7F17
:1009BB00131211BBE4FD7F071211BB7D907C167FD8
:1009CB00101211BB7D277C027F111211BB7F0A7E97
:1009DB00001211E67D9D7C007F121211BB7F0A7EF7
:1009EB00001211E67D007C197F131211BB7F0A7E6A
:1009FB00001211E67D257C007F291211BB7D0D7F36
:100A0B002B1211BB7D077F301211BB7403FDFC7FD2
:100A1B00311211BB7D037C007F321211BB7D067C32
:100A2B00027F351211BB7D087C007F361211BB7D16
:100A3B00067C047F371211BB7D041C7F381211BB5F
:100A4B007D077C007F391211BB7D027C067F3C1237
:100A5B0011BB7D087C007F3D1211BBE4FD7F501262
:100A6B0011BB7DEF7F511211BBE4FD7F521211BB05
:100A7B007D3F0C7F531211BB7D007CA77F60121151
:100A8B00BB7D017C007F611211BBE4FD7F6A1211FB
:100A9B00BBE4FD7F801211BBE4FD7F811211BBE42F
:100AAB00FD7F821211BBE4FD7F831211BBE4FD7F3E
:100ABB00841211BBE4FD7F851211BB7D107F901258
:100ACB0011BB7D007C067F921211BB7D337C017FB5
:100ADB00071211BB7D221CE4FF1211BB90020074A4
:100AEB0001F0A37440F0900216E4F0A374F0F07DD3
:100AFB00387C107F031211BBE4FDFC7F010211BB9C
:100B0B00900224ECF0A3EDF0A3EAF0A3EBF090023B
:100B1B0022EEF0A3EFF090022FEEF0A3EFF0E4A3A0
:100B2B00F090022AE0FBA3E0FAA3E0F9120854705C
:100B3B0003020C95900231E06003020C7690022DBB
:100B4B00E0FFC313FDC3900201E09DFD900200E0A6
:100B5B009400FCD3900223E09D900222E09C400382
:100B6B00020C95C3900217E09FFF900216E09400D1
:100B7B00FED3900225E09F900224E09E4003020CDE
:100B8B0095120854FF7E00D39480748094804008A3
:100B9B009002317401F08089EF640D4E702E90023B
:100BAB002DE0FF900225E02FF0900224E03400F0BE
:100BBB0090022FE0FFA3E0900222CFF0A3EFF09082
:100BCB00022BE475F00112089A020C6990022DE0D9
:100BDB00D3941074809480900222E0FE4038A3E0FE
:100BEB00FFA3E0FCA3E0FD900228E0FBA3E0900252
:100BFB0038CBF0A3EBF090022AE0FBA3E0FAA3E0E2
:100C0B00F912085490023AF0A374101205449002A2
:100C1B0023E024088040A3E0FFA3E0FCA3E0FD90C9
:100C2B000228E0FBA3E0900238CBF0A3EBF090029C
:100C3B002AE0FBA3E0FAA3E0F912085490023AF081
:100C4B0090022DE090023B12054490022DE0C3135D
:100C5B00FF900223E02FF0900222E03400F090028C
:100C6B002BE475F00112089A020B2C90022BE47501
:100C7B00F00212089A90022DE0FF900223E02FF071
:100C8B00900222E03400F0020B2C2278187C027DBB
:100C9B00017BFF7A1C798D7E007F0A12082E900251
:100CAB0000E0FAA3E0FB900216E0FFA3E09002281D
:100CBB00CFF0A3EFF074FFA3F0120DAB30B4FD43F4
:100CCB00BA8090FA737401F053BA7F121219900222
:100CDB002574FFF0A37412F0A37421F0A3EEF0A31C
:100CEB00EFF07B017A02791812024490022874FF0C
:100CFB00F0A374E0F0A37401F0A37402F0A37418D2
:100D0B00F0A37410F0A37401F07B1F7A007D197CA3
:100D1B00007F327E00120B0B43BA8090FA7374FF84
:100D2B00F053BA7F7F207E031211E6900200E0FAA7
:100D3B00A3E0FB900216E0FFA3E0900228CFF0A304
:100D4B00EFF0A374F8F0A3E4F0120DAE7F207E0356
:100D5B001211E6900200E0FAA3E0FB900216E0FF0E
:100D6B00A3E0900228CFF0A3EFF0A37407F074E098
:100D7B00120DAB7F207E031211E6900200E0FAA366
:100D8B00E0FB900216E0FFA3E0900228CFF0A3EF68
:100D9B00F0A3E4F0741F120DAB7F207E030211E66B
:100DAB00A3F0E4FDFCFFFE900222EEF0A3EFF0A314
:100DBB00ECF0A3EDF0900222E0FEA3E0FFC3EB9F6B
:100DCB00FFEA9ECF2401CF340090022EF0A3EFF068
:100DDB00900224E0FEA3E0FFC3900229E09FFF9066
:100DEB000228E09ECF2401CF3400900230F0A3EF15
:100DFB00F0900224E0FCA3E0FD900228E0FFA3E0CA
:100E0B00900248CFF0A3EFF0900222E0FEA3E0FFA8
:100E1B00120EF0E490022CF0A3F0FDFC90022AE0FD
:100E2B00FAA3E0FBED25E0FFEC33FE74002FF58217
:100E3B0074003EF583EAF0A3EBF00DBD00010CE46A
:100E4B00B505D9ECB401D59002127402F0A3745815
:100E5B00F0C2B443BA8090FA71E044A0F053BA7F69
:100E6B002243BA8090FE53E4F090000112086D64A7
:100E7B000190FE507006E04401F08004E054FEF057
:100E8B0090000212086D640290FE507006E044025E
:100E9B00F08004E054FDF090000312086DFFD39432
:100EAB000774809480500EEF25E025E0FF90FE51F3
:100EBB00E054E34FF090000412086DFFD3940374D9
:100ECB00809480500890FE51E054FC4FF01208546F
:100EDB00640190FE527006E04480F08004E0547F81
:100EEB00F053BA7F22900242EEF0A3EFF0AE04AFC4
:100EFB000590024AEEF0A3EFF0900248E0FFA3E06A
:100F0B0090024ECFF0A3EFF0900242E0FFA3E090EF
:100F1B00024CCFF0A3EFF0AF03900250EAF0A3EF37
:100F2B00F07F501211BB90024EE0FCA3E0FD7F510D
:100F3B001211BB7F521211B3900250E0FCA3E0FDE3
:100F4B007F531211BB90024AE0FCA3E0FD7F2012FD
:100F5B0011BB7F211211B37F2202113443BA80904F
:100F6B00FA72E4F09000011208B0FF90FA77E5F006
:100F7B00F0A3EFF09000031208B0FF90FA75E5F0C4
:100F8B00F0A3EFF090000512086D90FA73F01208C1
:100F9B0054640190FA717006E04480F08004E054D0
:100FAB007FF053BA7F2243BA8090FA70E054F0F08E
:100FBB00EDD3940374809480500BE0FEED25E02577
:100FCB00E0FDEE4DF0EBD3940374809480500690CB
:100FDB00FA70E04BF0EF640190FA707006E0448019
:100FEB00F08004E0547FF053BA7F7F002243BA8035
:100FFB0090FE54EFF053BA7FC2B4D20943BA80903B
:10100B00FE52E054F84484F053BA7F2009FD43BAF2
:10101B008090FE54EDF053BA7FD20943BA8090FE14
:10102B0052E054F84484F053BA7F2009FDD2B42225
:10103B0043BA8090FE54EFF053BA7FC2B4D2094347
:10104B00BA8090FE52E054F84485F053BA7F2009E1
:10105B00FD43BA8090FE54EDF053BA7FD20943BAE8
:10106B008090FE52E054F84485F053BA7F2009FD7E
:10107B00D2B42243BA8090FE50E054CFF0EDD3941B
:10108B000374809480500AE0FEEDC454F0FDEE4DE5
:10109B00F0EF640190FE507006E04480F08004E0B5
:1010AB00547FF053BA7F7F00227595007596FF53DE
:1010BB00B10F43B2F053B3FD43B40243BA8090FE79
:1010CB0051E0549F4420F053BA7F43BA8090FE50B6
:1010DB00E054F3F053BA7F22AB07AA068D828C83C0
:1010EB00C006C007AE83AF82900248EEF0A3EFF0CC
:1010FB00D007D006120EF0900214E0FEA3E0FF0220
:10110B001210EFB40A07740D121118740A309811EB
:10111B00A899B8130CC2983098FDA899C298B81129
:10112B00F63099FDC299F5992243BA8090FE54EF9F
:10113B00F053BA7FC2B4D20943BA8090FE52E05446
:10114B00F84484F053BA7F2009FDD2B422900218E0
:10115B007401F0E4A3F0A3F0A37402F0A314F0FB6A
:10116B007A027918120E6CE4FD7F0102107EC2B474
:10117B00D20A43BA8090FA71E04488F053BA7F20C8
:10118B000AFDD2B4900202E0FEA3E0FF22D2B47FAC
:10119B00327E001211E6C2B57F967E001211E6D2A6
:1011AB00B57F327E000211E690024CE0FCA3E0FD1D
:1011BB00AB05AA04AD07E4FF120FF8EAFFAD03027B
:1011CB00103B4202140000500202001100220033B7
:1011DB0000440055006600770088007DA37C08ED75
:1011EB001D70011C144C70F7EF1F70011E144E7014
:1011FB00EA221210B41211581200FAD2AF1209409F
:10120B00120C9680FBAD07AC06ECFF02103BE4FF23
:10121B0012113402117949443A30782578000000D4
:10122B0000000000000000000000000004040404A3
:10123B0004040004000000140A0A0000000000006F
:10124B000000000014143F140A3F0A0A00000004B7
:10125B001E1505060C14150F0400000012150D0ABF
:10126B00142C2A1200000000040A0A1E1515093658
:10127B00000000020201000000000000000000203E
:10128B0010080808080808102000000204080808C5
:10129B0008080804020000000004150E0E150400D7
:1012AB00000000000404041F0404040000000000FC
:1012BB000000000000000002020100000000001FFF
:1012CB000000000000000000000000000000000211
:1012DB0000000010080808040402020201000000CC
:1012EB000E1111111111110E00000000040604045F
:1012FB000404040E000000000E1111080402011F6B
:10130B00000000000E11100C1010110E0000000058
:10131B00080C0A0A091E0818000000001F01010F23
:10132B001010110E000000000E09010F1111110E0B
:10133B00000000001F09080404040404000000005E
:10134B000E11110E1111110E000000000E111111D2
:10135B001E10120E0000000000000400000000042C
:10136B000000000000000004000000040400002046
:10137B0010080402040810200000000000001F00E9
:10138B00001F0000000000020408102010080402D7
:10139B00000000000E1111080404000400000000FE
:1013AB000E111915151D011E0000000004040C0A76
:1013BB000A1E1233000000000F12120E1212120F2F
:1013CB00000000001E1101010101110E00000000C0
:1013DB000F1212121212120F000000001F120A0E2F
:1013EB000A02121F000000001F120A0E0A02020757
:1013FB00000000001C1201013911120C000000004A
:10140B003312121E12121233000000001F040404C8
:10141B000404041F000000003E080808080808091F
:10142B000700000037120A060A0A123700000000F4
:10143B00070202020202223F000000001B1B1B1BC3
:10144B0015151515000000003B1216161A1A121767
:10145B00000000000E1111111111110E00000000FF
:10146B000F12120E02020207000000000E111111E2
:10147B001117190E180000000F12120E0A12123754
:10148B00000000001E1101060810110F00000000E3
:10149B001F1504040404040E000000003312121282
:1014AB001212120C000000003312120A0A0C040470
:1014BB00000000001515150E0A0A0A0A00000000AC
:1014CB001B0A0A04040A0A1B000000001B0A0A0478
:1014DB000404040E000000001F0908040402121F7C
:1014EB000000001C04040404040404041C00000297
:1014FB0002020404080808100000000E080808087F
:10150B00080808080E0000040A0000000000000094
:10151B00000000000000000000000000003F00047D
:10152B000000000000000000000000000000000CA4
:10153B00121C123C000000000302020E1212120ECB
:10154B00000000000000001C1202021C0000000042
:10155B001810101C1212123C000000000000000CAE
:10156B00121E021C000000003804041E0404041E9A
:10157B00000000000000003C120C021E221C0000A8
:10158B000302020E121212370000000004000006C4
:10159B000404040E000000000800000C08080808F2
:1015AB00080700000302023A0A0E1237000000007F
:1015BB00070404040404041F000000000000000FD3
:1015CB0015151515000000000000000F1212123740
:1015DB00000000000000000C1212120C00000000B2
:1015EB000000000F1212120E020700000000001C78
:1015FB001212121C103800000000001B060202071A
:10160B00000000000000001E020C101E0000000075
:10161B000004040E04040418000000000000001B6A
:10162B001212123C0000000000000037120A0C04DA
:10163B000000000000000015150E0A0A0000000053
:10164B000000001B0A040A1B00000000000000370A
:10165B00120A0C04040300000000001E0804041E00
:10166B0000000018080808040808080818000808F3
:10167B0008080808080808080808000604040408F5
:10168B0004040404060002251800000000000000FA
:10169B00000000000000000000000000000000003F
:1016AB0000000000000808080808080800001818C7
:1016BB00000000486C241200000000000000000035
:1016CB0000000000002424247F1212127F12121239
:1016DB0000000000081C2A2A0A0C1828282A2A1C99
:1016EB00080800000022251515152A5854545422B9
:1016FB0000000000000C1212120A76252911916EBF
:10170B0000000006060403000000000000000000BB
:10171B0000000040201010080808080808101020CE
:10172B0040000002040808101010101010080804E4
:10173B0002000000000008086B1C1C6B080800006E
:10174B00000000000000080808087F0808080800CF
:10175B000000000000000000000000000000060672
:10176B0004030000000000000000FE000000000069
:10177B000000000000000000000000000000060652
:10178B0000000000804040202010100808040402D4
:10179B0002000000001824424242424242422418F6
:1017AB000000000000080E08080808080808083E9A
:1017BB0000000000003C4242422020100804427E00
:1017CB0000000000003C4242201820404042221CF6
:1017DB000000000000203028242422227E202078C4
:1017EB0000000000007E0202021A26404042221C2A
:1017FB000000000000382402021A2642424224183C
:10180B0000000000007E22221010080808080808BB
:10181B0000000000003C4242422418244242423C59
:10182B000000000000182442424264584040241C2F
:10183B00000000000000000018180000000018183D
:10184B00000000000000000000080000000000087D
:10185B000804000000402010080402040810204077
:10186B0000000000000000007F0000007F0000006F
:10187B0000000000000204081020402010080402A1
:10188B0000000000003C4242464020101000181897
:10189B0000000000001C225A555555552D42221CA4
:1018AB0000000000000808181414243C224242E7F0
:1018BB0000000000001F2222221E22424242221F51
:1018CB0000000000007C4242010101010142221C88
:1018DB0000000000001F2242424242424242221FAD
:1018EB0000000000003F4212121E12120242423F41
:1018FB0000000000003F4212121E121202020207E9
:10190B0000000000003C2222010101712122221C57
:10191B000000000000E7424242427E42424242E760
:10192B0000000000003E0808080808080808083EE8
:10193B0000000000007C1010101010101010101080
:10194B00110F0000007722120A0E0A1212222277C0
:10195B000000000000070202020202020202427FA4
:10196B00000000000077363636362A2A2A2A2A6BE0
:10197B000000000000E346464A4A52525262624758
:10198B0000000000001C2241414141414141221C09
:10199B0000000000003F424242423E0202020207A8
:1019AB0000000000001C2241414141414D53321CBB
:1019BB0060000000003F4242423E1212222242C708
:1019CB0000000000007C4242020418204042423ECC
:1019DB0000000000007F4908080808080808081CD8
:1019EB000000000000E74242424242424242423C77
:1019FB000000000000E742422224241414180808B7
:101A0B0000000000006B49494949555536222222F6
:101A1B000000000000E7422424181818242442E791
:101A2B000000000000772222141408080808081C84
:101A3B0000000000007E2120101008040442423FE9
:101A4B0000000078080808080808080808080808B3
:101A5B00780000000202040408080810102020205F
:101A6B004040001E1010101010101010101010100D
:101A7B001E000038440000000000000000000000C1
:101A8B00000000000000000000000000000000004B
:101A9B0000FF00060800000000000000000000002E
:101AAB000000000000000000003C4278444242FC71
:101ABB000000000000030202021A26424242261ACC
:101ACB00000000000000000000384402020244380D
:101ADB00000000000060404040784442424264D81D
:101AEB000000000000000000003C427E0202423C6D
:101AFB000000000000F08808087E08080808083E6F
:101B0B000000000000000000007C22221C023C426E
:101B1B00423C000000030202023A4642424242E7C4
:101B2B0000000000000C0C00000E08080808083E1E
:101B3B000000000000303000003820202020202042
:101B4B00221E0000000302020272120A16122277F2
:101B5B0000000000000E0808080808080808083EE6
:101B6B000000000000000000007F9292929292B75A
:101B7B000000000000000000003B4642424242E7EA
:101B8B000000000000000000003C42424242423C88
:101B9B000000000000000000001B26424242221EF3
:101BAB0002070000000000000078444242424478E3
:101BBB0040E000000000000000774C040404041F08
:101BCB000000000000000000007C42023C40423E4E
:101BDB000000000000000008083E08080808083054
:101BEB00000000000000000000634242424262DC41
:101BFB00000000000000000000E742242414080845
:101C0B00000000000000000000EB4949555522225E
:101C1B000000000000000000007624181818246E45
:101C2B00000000000000000000E742242414180804
:101C3B000807000000000000007E22100808447E08
:101C4B00000000C020202020201020202020202059
:101C5B00C0001010101010101010101010101010D9
:101C6B0010100006080808080810080808080808DB
:101C7B0006000C32C2000000000000000000000053
:0C1C8B000000000000000000000000004D
:00000001FF
